:1000000001308A0077290000D3346D38EC32202A81
:10001000E832F236EF36653AE8327210A0060A008E
:10002000CC224410253658100D050000D63C7336FE
:100030006532EE3220265321A0126C2CA0060A0055
:1000400083168611831286110830F80027280000D5
:10005000F8173828F813AF0C03188615031C8611FF
:10006000781738287813F80B2B28362800008615C7
:100070003F308400840B3A280000F81B2A28781BA4
:1000800032280800831603178C170C140000000098
:1000900083120C087F39031986280313AB0003175A
:1000A0000D080313AC0003170F080313AD002B0852
:1000B000AF0020202C0803178D0003132D08031711
:1000C0008F0083168C170C140000000083120C0D97
:1000D0000E0D7F39031986280313AB0003170D0893
:1000E0000313AC0003170F080313AD002B08AF0078
:1000F00020202C0803178D0003132D0803178F00F1
:100100008D0A03198F0A03134228031703138A1158
:100110000A12DF290830F8000000861083168610C6
:1001200000008312AB0D0610031C992883160614D9
:10013000831203189E2883160610831283168614D2
:100140008312861CA128F80B8C28000086108316C9
:100150008610000006140000000086148312861C1E
:10016000AF28F80100000618781486108316861050
:100170008312061083160610831208002B308400A9
:10018000831300080319D1280230F800F701F70B98
:10019000C728F80BC6289730F700F70BCD28800B3F
:1001A000C42808000830AC007708AD008316061498
:1001B000000086148312861CDB2806180314061C14
:1001C0000310F80D00008316861083128610AC0B06
:1001D000D628831606140000831206102D08031972
:1001E000F4288316061083120000831686148312E7
:1001F000861CF828000086108316861000008312E3
:1002000006108316061083128A110A12C12A831659
:1002100003178C170C1400000000031836298312F2
:100220000C087F390313AC0003170D080313AD004E
:1002300003170F080313AE002C08AF0020202D0871
:1002400003178D0003132E0803178F0083168C17D6
:100250000C140000000083120313AB0B3029332968
:1002600083160317362955298316031783120C0D9D
:100270000E0D7F390313AC0003170D080313AD00F7
:1002800003170F080313AE002C08AF0020202D0821
:1002900003178D0003132E0803178F008D0A03190F
:1002A0008F0A03100313AB0B07290800AC1B682946
:1002B0000F30F7002B0EF7050A3077020318632979
:1002C0003030F70765292C08F7077708AF002020A2
:1002D0000F30AB050A302B02031870293030722919
:1002E000AC132C08AB072B08AF00202008008401BA
:1002F00083131F308305713083168F000F0886111A
:1003000083128615831603170908C0398900031361
:100310001F129F1200300317880083128701880183
:100320008901FF300313A000831603170908C039A1
:10033000890003131F129F120030031788008312D5
:1003400003131F139F1383169F1383121F149412FA
:10035000A012200883168700831220162008831617
:1003600087008312A01120088316870001308312B2
:1003700094000030831694000108C73908388100C2
:10038000831290010030F800920000308316920032
:100390008312201520088316870083129701831685
:1003A0009B019C0101309D00831203178701880186
:1003B000890104308D0000308F0003134228A7010B
:1003C000A90183160614000086140000831206108B
:1003D0008316061000008312861083168610AA303A
:1003E0008312AB008A206130AB008A20831606148A
:1003F0000000861400008312861CFC290610831658
:10040000061000008312861083168610AA3083120D
:10041000AB008A20AB018A208316061000008614E8
:100420008312861C112A0000152A00008316061468
:10043000000001308312AB00BE20831606140000BA
:100440008614000083120610831606100000831223
:10045000861083168610AA308312AB008A203E30A5
:10046000AB008A2083160614000086140000831255
:10047000861C382A06108316061000008312861088
:1004800083168610AA308312AB008A204030AB005E
:100490008A2083160610000086148312861C4E2ABA
:1004A0000000522A00008316061400000130831257
:1004B000AB00BE20831606140000861400008312D1
:1004C000061083160610000083128610831686100D
:1004D000AA308312AB008A203F30AB008A208316FB
:1004E00006140000861400008312861C752A06106C
:1004F0008316061000008312861083168610AA3019
:100500008312AB008A20AB018A20831606100000FC
:1005100086148312861C8A2A00008E2A0000831605
:100520000614000001308312AB00BE2083160614AF
:1005300000008614000083120610831606100000C7
:100540008312861083168610AA308312AB008A208D
:100550004430AB008A208316061400008614000085
:100560008312861CB12A061083160610000083121F
:10057000861083168610AB308312AB008A20F701F9
:10058000D2287808A800831606100000861483126B
:10059000861CC82A0000CC2A00008316061400001E
:1005A00001308312AB00BE20103003178D000030E5
:1005B0008F00031004300313AB0007212808AB00A1
:1005C0003730AC0056212030AF0020200D30AF0076
:1005D00020200A30AF0020202808533C031D0C2B9C
:1005E0000130A702163003178D0000308F00031072
:1005F0000D300313AB0007212708AB003730AC00E8
:1006000056212030AF0020200D30AF0020200A30CE
:10061000AF0020200A2B862B8316061400008614B8
:100620000000831206108316061000008312861045
:1006300083168610AA308312AB008A204430AB00A8
:100640008A20831606140000861400008312861C7C
:10065000272B0610831606100000831286108316BF
:100660008610AA308312AB008A205330AB008A2058
:1006700083160610000086148312861C3D2B000092
:10068000412B000083160614000040308312AA009C
:10069000A401A301A601A501831606140000861477
:1006A00000008312061083160610000083128610C5
:1006B00083168610AA308312AB008A206030AB000C
:1006C0008A20831606140000861400008312861CFC
:1006D000672B0610831606100000831286108316FF
:1006E0008610AA308312AB008A202708AB008A202C
:1006F00083160610000086148312861C7D2B0000D2
:10070000812B000083160614000083120130A70716
:0A0710006430AB00BE20E129630055
:04400E00F52CFF3F4F
:00000001FF
